:020000040000FA
:06000000D2EF03F0120034
:06000800A2EF00F012005F
:06001800C7EF00F012002A
:06002A000100E2070000E6
:080030000000000024000000A4
:0800380013D87BD8BDD887D98D
:10004000CD80D180F2D914DA6EDA8DDABCDA3C5088
:1000500002E0F0DA3C6AE8DA03000000F3D71200AD
:10006000C20ED36EC76A300EC66E0B0EC16E0F0E77
:10007000926E440E936E800E946E800E956E020EFC
:10008000966E806A816A826A200E836E846A200E70
:10009000C96ED40E246E300E256E2406000E255A2D
:1000A0002450251003E000000000F7D7D09C3C0E40
:1000B0002C6E4E0ECD6ECF68CE689D909E90346AA9
:1000C000356A010E366E386A100E396E3A6A8484CB
:1000D000020E246E256A2406000E255A245025108F
:1000E00003E000000000F7D78150040B02E0F19814
:1000F00001D0F188F088F08EF092010E3B6E9ADA12
:10010000C40E246E090E256E2406000E255A2450B6
:10011000251003E000000000F7D73B6A070EB16E20
:10012000A082A292A192B190D08EF28CF28E3C6A03
:100130001200900EAB6E240EAC6E0C0EAF6E380E2D
:10014000B86E1200DACFE4FFE6528480F092845059
:10015000020B01E0010E4E6EF150100B01E0010E9A
:100160004E5C07E10F0E395C02E3396A08D0392A88
:1001700006D0395003E10F0E396E01D03906849054
:10018000F178010E3A6EE552E5CFDAFF1100D8CFD3
:10019000E4FFE0CFE4FFE46EDACFE4FFE652010EC5
:1001A0003B6EB190A192E552E5CFDAFFE550E5CF85
:1001B000E0FFE5CFD8FF10008386839495940D0E61
:1001C000246E256A2406000E255A2450251003E0CB
:1001D00000000000F7D7958417D8000904E1838850
:1001E000030000000ED0330E2A6E23D8100E2E6EA0
:1001F0002E50000805E247D865D8020E2E5EF8D7CB
:1002000089D8958483861200030E246E256A2406FD
:10021000000E255A2450251003E000000000F7D7F7
:1002200083B404D083A4FED7010E02D0000E00D008
:1002300012002D6A2D50070825E32AA010D08394C0
:1002400095949584020E246E256A2406000E255A84
:100250002450251003E000000000F7D70FD083944E
:100260009594020E246E256A2406000E255A245009
:10027000251003E000000000F7D795842A902A4259
:100280002D2AD8D712002B6A2D6A2D50070819E3A2
:100290002B902B428394959495840000000083A4B6
:1002A00002D0800E2B26030E246E256A2406000E33
:1002B000255A2450251003E000000000F7D72D2A0E
:1002C000E4D712002B380F0BF76AC00FF66E070E3B
:1002D000F7220800F550E66E020E2E5CEA6A130F54
:1002E000E96E000EEA22E552E750EF6E0F0E2B1476
:1002F000F76AC00FF66E070EF7220800F550E66E9B
:100300002E04EA6A130FE96E000EEA22E552E75066
:10031000EF6E12000D0EAD6EACA2FED72D6A100E60
:100320002D5C0CE22D50EA6A130FE96E000EEA22F2
:10033000EF50AD6EACA2FED72D2AF1D70D0EAD6EEB
:10034000ACA2FED70A0EAD6EACA2FED71200838817
:10035000A80E246E610E256E2406000E255A245028
:10036000251003E000000000F7D7839863D9A80E9A
:10037000246E610E256E2406000E255A2450251089
:1003800003E000000000F7D74F0E006E4F0E016E25
:100390004F0E026E4F0E036E4F0E046E4F0E056E23
:1003A0004F0E066E4F0E076E4F0E086E43D9A80E05
:1003B000246E610E256E2406000E255A2450251049
:1003C00003E000000000F7D7110E006E110E016E61
:1003D000110E026E110E036E110E046E110E056EDB
:1003E000110E066E110E076E110E086E23D9A80E9F
:1003F000246E610E256E2406000E255A2450251009
:1004000003E000000000F7D7010E3B6E13D9A80EE1
:10041000246E610E256E2406000E255A24502510E8
:1004200003E000000000F7D7120083989EA01FD0C1
:10043000F29ECE50336ECE50335CFDE0800ECF2660
:100440009E90F28E342A640E345C02E1346A356A7E
:100450003450266E0BD928500C6E29500D6E010EAB
:100460003C6E352A0A0E355C02E1356A838812003B
:100470002C2A3F0E2C5C56E12C6A838C1B0EC16E1D
:10048000090EC06E010E246E256A2406000E255A40
:100490002450251003E000000000F7D7070EC26EBD
:1004A000C2B2FED7839CC290C3CF2FF0C4CF30F02E
:1004B000316A326AD40E476E486A496A4A6A2FC066
:1004C00042F030C043F031C044F032C045F09AEC05
:1004D00003F03EC02FF03FC030F040C031F041C0CB
:1004E00032F030C02FF031C030F032C031F0326A1B
:1004F00030C02FF031C030F032C031F0326A100E0F
:100500002F26000E3022000E3122000E32222F50F4
:10051000266EACD82850096E29500A6E3F0E0B6E1D
:10052000010E3C6E12009EAA1DD03B6AAE50006EBA
:10053000AE50016EAE50026EAE50036EAE50046E01
:10054000AE50056EAE50066EAE50076EAE50086EE1
:10055000010E3C6EB190B26AB36AB180AE50AD6E1E
:10056000ACA2FED712003850382A4F6E060E4F5CF0
:1005700029E3386A3650376E0B0EC16E090EC06E15
:10058000808E030EC26EC2B2FED7809EC290C4504F
:10059000366E3750365C16E036380F0BF76AC00FF0
:1005A000F66E070EF7220800F5500F6E0F0E361488
:1005B000F76AC00FF66E070EF7220800F550106EAE
:1005C000010E3C6E12003A502EE03A6A0F0E3914BA
:1005D000F76AC00FF66E070EF7220800F550AD6EF1
:1005E000ACA2FED70D0EAD6EACA2FED70A0EAD6E5C
:1005F000ACA2FED73B6A3950006E3950016E3950BB
:10060000026E3950036E3950046E3950056E395000
:10061000066E3950076E3950086E010E3C6EB1906F
:10062000B26AB36AB18012008480000083AE83880E
:1006300084901200839A2D6A2D50080815E39E9627
:100640003B5006E02D50EA6A090FE96E000E05D016
:100650002D50EA6A000FE96E000EEA22EF50C96ED3
:100660009EA6FED72D2AE8D7838A1200300E276E69
:10067000286E296E640E265C04E3272A640E265E2B
:10068000F9D70A0E265C04E3282A0A0E265EF9D75B
:060690002650292612008D
:0A0696002A0EF66E000EF76E000E3D
:1006A000F86E00010900F550856F0900F550866F5E
:1006B00003E1856701D03DD00900F550806F090046
:1006C000F550816F0900F550826F09000900F5505F
:1006D000E96E0900F550EA6E090009000900F550BD
:1006E000836F0900F550846F09000900F6CF87F089
:1006F000F7CF88F0F8CF89F080C0F6FF81C0F7FF10
:1007000082C0F8FF0001835302E1845307E009002F
:10071000F550EE6E8307F8E28407F9D787C0F6FF3D
:1007200088C0F7FF89C0F8FF00018507000E865BCF
:04073000BFD712001D
:0C07340042504702F3CF3EF0F4CF3FF0FC
:100740004802F3503F26000EF420406E425049020A
:10075000F3504026000EF420416E42504A02F350FE
:10076000412643504702F3503F26F4504022000EEA
:10077000412243504802F3504026F4504122435056
:100780004902F350412644504702F3504026F450AA
:10079000412244504802F350412645504702F3504D
:0407A00041261200DC
:0C07A40011EE00F021EE00F0F86A4D9C10
:1007B0004BEC03F0F0EC03F01CEC00F0FBD7120064
:1007C0003031323334353637383941424344454687
:0107D0000028
:0E07D20000EE00F00F0EEE6AEA62FDD7120094
:0207E000120005
:0E07E2001010101010101010102020202020D9
:1007F0002020202000202020202020202020202019
:0608000020202020200052
:020000040030CA
:0100010009F5
:010002001AE3
:0100030004F8
:01000500807A
:010006008178
:0100080003F4
:01000900C036
:01000A0003F2
:01000B00E014
:01000C0003F0
:01000D0040B2
:00000001FF
